:100000000CC027C026C025C024C023C022C021C0E8
:1000100020C01FC01EC01DC01CC011241FBECFE5C4
:10002000D2E0DEBFCDBF10E0A0E6B0E0E6EDF0E04C
:1000300003C0C89531960D92A036B107D1F710E0F4
:10004000A0E6B0E001C01D92A036B107E1F710D0E4
:1000500041C0D6CFCF93DF93CDB7DEB7E8E3F0E072
:100060001082E7E3F0E081E08083DF91CF91089593
:10007000CF93DF93CDB7DEB722970FB6F894DEBFEC
:100080000FBECDBFE7DFE6E3F0E080819927817006
:100090009070882349F0A8E3B0E0E8E3F0E09081B5
:1000A0008EEF89238C9307C0A8E3B0E0E8E3F0E08B
:1000B000808181608C9380E593EC9A83898305C06D
:1000C00089819A8101979A83898389819A8100978E
:0600D000B9F7D9CFFFCF04
:00000001FF
